:100000000C9436040C946E040C946E040C946E04E0
:100010000C946E040C946E040C946E040C946E0498
:100020000C946E040C946E040C9445300C941D31A9
:100030000C94FA2F0C946E040C946E040C946E04C1
:100040000C946E040C946E040C946E040C946E0468
:100050000C946E040C9421300C946E040C946E0479
:100060000C946E040C946E040C946E040C946E0448
:100070000C946E040C946E040C946E040C946E0438
:100080000C946E040C946E040C946E040C946E0428
:100090000C946E040C946E040C946E040C946E0418
:1000A0000C946E040C946E040C946E04050109808B
:1000B000A101850319012AB700150126B700950192
:1000C00075108100C0050C0901A101850419012AE0
:1000D000A002150126A002950175108100C00660DE
:1000E000FF0961A1010962150026FF00952075082E
:1000F00081020963150026FF00952075089102C052
:1001000005010906A101050719E029E715002501E8
:10011000950875018102950175088101050719008F
:1001200029FF150026FF00950675088100050819AE
:10013000012905950575019102950175039101C08D
:100140000E018466FFFF000000000F018466FFFFC0
:100150000000000010018466FFFF000000000301A2
:100160008466FF0A0155FFFF120155FFFFFF0000E3
:10017000000004018466FF090155FFFF130155FFCC
:10018000FFFF0000000011018466FF180155FFFF0A
:10019000FF000000000B018466FFFF000000001458
:1001A000018466FF0C0155FFFFFF00000000000006
:1001B000000000000000000000000000000000003F
:1001C000000000000000000000000000000000002F
:1001D00000007E0F00D4FFFFFFC700000078000082
:1001E0000000000000002A2B280000000000000092
:1001F00000000000000000000029000000002C1E8C
:100200003420212224342627252E362D3738271E48
:100210001F202122232425263333362E37381F046E
:1002200005060708090A0B0C0D0E0F101112131406
:1002300015161718191A1B1C1D2F3130232D3504C4
:1002400005060708090A0B0C0D0E0F1011121314E6
:1002500015161718191A1B1C1D2F3130354C0902A1
:100260005B00030100A0FA09040000010301010082
:100270000921110100012240000705810308000146
:1002800009040100020300000009211101000122FC
:100290002200070582032000010705030320000157
:1002A00009040200010300000009211101000122DC
:1002B0003200070584032000011201000200000043
:1002C00008F1F125000100010203011C0376006919
:1002D0000061006C003A00660036003400630032B2
:1002E0000062003300630000001603570069006ECF
:1002F00000720079002000320035007400660000B2
:10030000001A035300700069006400650072004920
:100310000073006C0061006E0064000000040309BB
:1003200004530054005500560029005F006000612E
:10033000005700C25C5C005D005E005800C35C5961
:10034000005A005B005200015162006300500051EE
:10035000004F00C25CC35CC45CCD5CC55CC95CC7BB
:100360005CC55CCB5CCE5CCA5CC85CC65CCC5C002B
:1003700000025303530453000000000553065307C3
:10038000530000000000000000000000000000001A
:100390000000005A00000000000000000000000003
:1003A00000000000000000000000000050000000FD
:1003B000000000000000000000000000000000003D
:1003C00000000000005B00000000000000000000D2
:1003D00000000000000000000000000000005000CD
:1003E000000000000000000000000000000000000D
:1003F000000000000000005C0000000000000000A1
:1004000000000000000000000000000000000000EC
:10041000500000000000000000000000000000008C
:100420000000000000000000005D0000000000006F
:1004300000000000000000000000000000000000BC
:10044000000050000000000000000000000000005C
:1004500000000000000000000000005E000000003E
:10046000000000000000000000000000000000008C
:10047000000000005000000000000000000000002C
:10048000000000000000000000000000005F00000D
:10049000000000000000000000000000000000005C
:1004A00000000000000050000000000000000000FC
:1004B000002223252628292A2C2D2F3032333536A9
:1004C000383A3B3D3E4042434547494A4C4E5051E5
:1004D000535557595A5C5E6062646668696B6D6F0C
:1004E00071737577797B7D7F81838587898A8C8E0F
:1004F00090929496989A9C9E9FA1A3A5A7A8AAAC17
:10050000AEAFB1B3B4B6B8B9BBBCBEBFC1C2C3C550
:10051000C6C7C9CACBCCCDCED0D1D2D2D3D4D5D6F2
:10052000D7D7D8D9D9DADADBDBDBDCDCDCDCDCDD25
:10053000DDDDDDDCDCDCDCDCDBDBDBDADAD9D9D809
:10054000D7D7D6D5D4D3D2D2D1D0CECDCCCBCAC9A1
:10055000C7C6C5C3C2C1BFBEBCBBB9B8B6B4B3B1D0
:10056000AFAEACAAA8A7A5A3A19F9E9C9A9896946B
:1005700092908E8C8A89878583817F7D7B79777540
:1005800073716F6D6B6968666462605E5C5A59571F
:10059000555351504E4C4A4947454342403E3D3BDE
:1005A0003A3836353332302F2D2C2A292826252368
:1005B00022FFAA7F55400001010101010101010153
:1005C0000202020202020202020303030303030304
:1005D00003040404040404040505050505060606D1
:1005E0000606070707070708080808090909090A8E
:1005F0000A0A0B0B0B0C0C0C0D0D0D0E0E0E0F0F33
:100600000F101011111112121313141415151616C0
:100610001717181819191A1A1B1B1C1D1D1E1E1F2F
:100620002020212222232424252626272829292A7E
:100630002B2C2D2D2E2F30313232333435363738A6
:10064000393A3B3C3D3E3F404142434445464748A2
:10065000494A4C4D4E4F50515354555658595A5B78
:100660005D5E5F616264656668696B6C6D6F707218
:10067000737577787A7B7D7E8082838587888A8C84
:100680008E8F91939596989A9C9EA0A2A3A5A7A9B8
:10069000ABADAFB1B3B5B7BABCBEC0C2C4C6C9CBAF
:1006A000CDCFD1D4D6D8DBDDDFE2E4E7E9EBEEF065
:1006B000F3F5F8FAFDFF9F019501860172015E01D5
:1006C00054014A01400100001E0F057F3F1F6432A4
:1006D00014643214783C1E1E140A0501000100CB7C
:1006E00003F3280929000002000200C703F32809C8
:1006F00029000003000100CC03F3280929000004AD
:10070000000200B103F3280929DB0705000100CD31
:1007100003F3280929000006000200B303F32809A7
:1007200029000007000200C903F328092900000876
:10073000000100CE03F3280929000012000200CFB7
:1007400003F3280929000013000200D103F328094C
:1007500029000014000100D303F328092900001523
:100760000000000000E407610F0000FD377A585ACE
:10077000000004E6D6B44602002101160000007411
:100780002FE5A3E0016000C05D003D8889C65436B6
:10079000C3174FE4E881DCB77554611F8F0ADB9EF5
:1007A00081481ACFAD54ECECB46DFB7A059B70FE1A
:1007B00049D9CAA8592FBFB1C016AB2E04269E83B3
:1007C00071FC64ADC7A154C715F383E2A7CE12E153
:1007D000EF62AAB691F187EC8B70FF689B9FABE448
:1007E0009163D1B8395B705E5160692507F5D0EE31
:1007F000860A9E1D1EA97AA16D9BA0932B2439A069
:100800009B8C948FC8B59954A08FF6F4915BF244F9
:10081000F1AF3DE80066100254CE4967844A75C7BF
:10082000329D6B8A170CAE5C67275819908D59EA78
:10083000AEF8B67A01DB02B58876EF91E577E1B1E3
:10084000EA1BD0F4A310FD55D500004B0A2F270D4D
:10085000C9F2180001DC01E10200000AD38EF6B1F2
:10086000C467FB020000000004595A0011241FBE97
:10087000CFEFDAE0DEBFCDBF04B603FE18C0809133
:10088000D9039091DA03A091DB03B091DC038730A8
:10089000904BA740B04B59F41092D9031092DA0351
:1008A0001092DB031092DC03E0E0F8E3099523E00B
:1008B000A2EAB1E001C01D92A93DB207E1F711E043
:1008C000A0E0B1E0E4E6F7E602C005900D92A23A9E
:1008D000B107D9F70E94DF290C9457330C9400001C
:1008E0009C01FB019A9581159F4120F5D901AA270A
:1008F000B270832F8170B90166277470A9014427F3
:10090000587034FF0DC08295807FAB2B09F0806258
:10091000672B09F08064452B09F0806809950895DC
:10092000AB2B09F08260672B09F08460452BB1F393
:100930008860F4CF80E0F2CF282F92959F70963098
:1009400091F060F4925F9F70923030F481E0203F2C
:1009500079F030F4283E30F080E008959A5FF3CFCC
:10096000243FD1F7089581E0283EE0F3213FF9CFFD
:100970000895292F953098F5853088F590E035E079
:10098000239F800D911D1124282F277041E001C065
:10099000440F2A95EAF723E0969587952A95E1F783
:1009A000FC01EE0FFF1FE80FF91FE25DFC4F20E096
:1009B00030E070E05191DF011197CB01022E02C0AF
:1009C000969587950A94E2F781708195852784230F
:1009D00085278C932F5F3F4F2330310559F70895BA
:1009E000292F953078F5853068F590E035E0239F24
:1009F000800D911D1124682F677023E096958795CF
:100A00002A95E1F7FC01EE0FFF1FE80FF91FE25DE9
:100A1000FC4F40E050E080E0219130E0062E02C023
:100A2000369527950A94E2F721703327042E01C0EA
:100A3000220F0A94EAF7822B4F5F5F4F4330510534
:100A400059F7089580E0089580917A039091790391
:100A5000981301C008958F5F8770FACFE6EAF1E03E
:100A60009191891303C0DF0111971C9291E0EC3A38
:100A7000F907B1F70895982F909580917103892314
:100A800080937103089580917003882331F0109250
:100A9000700310922D0310922C0308959091D503AA
:100AA00092FF06C0282F28712830F9F4877F8460D0
:100AB00093FF06C0282F28712831F1F4877E8461C6
:100AC0002091D60320FF06C0382F38713830D9F472
:100AD000877F816021FF06C0282F28712831D1F43B
:100AE000877E816194FD877E0895282F24712430AC
:100AF000F9F68B7F8860DCCF282F2471243101F731
:100B00008B7E8861DDCF382F3171313019F78E7FC0
:100B10008860E0CF282F2171213121F78E7E8861F6
:100B2000E1CFCF93DF93EC01803E910509F47AC0C9
:100B300090F58133910509F4C0C088F4893291059C
:100B400009F4B0C08A32910509F4BEC0019709F4D6
:100B50007AC0CE010497813A9105D0F474C08933EC
:100B6000910509F453C08238910509F44FC08533CB
:100B7000910509F492C0883A910530F4853A9105BF
:100B800040F3A497D0645FC08F3B910508F4F3C095
:100B9000C0E0D0E058C0843E910509F463C0B0F4D1
:100BA000823E910509F44BC0833E910509F44FC084
:100BB000C11580E4D80708F0E9C0C83ED10508F4A3
:100BC00042C0CE019A958F3F9E41C7CF863E910588
:100BD00009F453C0873E910509F454C0811523E5FB
:100BE000920708F078C0811542E5940708F0E6C046
:100BF000811550E59507E0F2811561E5960708F447
:100C0000C8C0D82FCC27C16FD06A1DC08091D50332
:100C10008370811103C18091D60383FF14C0C9E2A0
:100C2000D0E011C08091D50380FD44C09091D603DF
:100C300090FF09C0C3EED0E084FDAACF04C080912C
:100C4000D50382FDF7CFCE01DF91CF91089580913A
:100C5000D50382FDE0C09091D60390FDDFC084FFF4
:100C6000F2CF96CF8091D60381FFEDCF8091D5034F
:100C7000C7EED0E084FD8CCFE6CF8091D50383FD15
:100C8000F7CFE1CF8091D50383FDCBC09091D60300
:100C900091FFE5CFC4EED0E0D6CF8091D50385FF9C
:100CA000D2CFBDCF8091D50385FDBEC08091D60344
:100CB00083FFC9CFC9E3D0E0C6CF8091D50386FFBB
:100CC000C2CFCAE2D0E0BFCF8091D50386FFBBCFB1
:100CD000C1E3D0E0B8CF811549E59407A8F58115A7
:100CE00058E5950708F084C0811565E59607D8F4A6
:100CF000C11584E5D80708F076C08C2F86958695B7
:100D000020E2829FC0011124C370DD2721E030E082
:100D1000A90102C0440F551FCA95E2F7EA01C82B8A
:100D2000D92BDA6890CF95558F3F910511F008F0D7
:100D30002FCF8C2F0E944E05C82FD0E0DC2FCC2760
:100D4000CC27DF71D0627FCFC1158AE5D80708F4C0
:100D500054C0CE0190568115904208F019CF8D2FC6
:100D60008F710E944E0590E0982F882788279F71E9
:100D70008C2BEC01E7CFC85AD0E0CC0FDD1FCD584B
:100D8000DE4F0990D881C02DD4645DCFDF70D06A6A
:100D90005ACF86958695837040E2849FC0011124C6
:100DA000C37021E030E0A90102C0440F551FCA956D
:100DB000E2F7EA01C82BD92BDD6845CF86958695E9
:100DC00050E2859FC0011124C370DD2721E030E08F
:100DD000A90102C0440F551FCA95E2F7EA01C82BCA
:100DE000D92BDC6830CFDC2FCC27C46FD06A2BCF57
:100DF000D82FCC27C06FD06A26CF8C2F8F700E943F
:100E00004E0534E0D695C7953A95E1F7CF709C2F03
:100E1000EC01D06918CFC2EED0E015CFC0EED0E023
:100E200012CFC6EED0E00FCFC5E3D0E00CCF80E00C
:100E30000895F894E82FE295EF70F0E041A18F70EB
:100E400021E030E0B90102C0660F771F8A95E2F712
:100E5000CB01962F9095942391A392A1892B82A3E5
:100E6000789408950895A0E0B0E0E9E3F7E00C94E9
:100E7000CC31E901E42FF0E0EA54FA4F61110BC0E4
:100E8000E4919E2F8E2F8983E8839A83CDB7DEB7B6
:100E9000EAE00C94E831282F30E0062F10E0F491BE
:100EA000EF2F86E0829F6001839FD00C1124EE24F7
:100EB000EA94F12CC601B7010E948031220F331F42
:100EC00045E5469FC001479F900D1124281B390B13
:100ED000822F880F280FC701801B910BF89FA0015C
:100EE000F99F500D1124952F209F5001219FB00C88
:100EF0001124AB2CBB24D701AA19BB095D01FA9DB3
:100F0000D001FB9DB00D11248B2F5701A21AB108FF
:100F10009501209F5001219FB00C309FB00C1124EF
:100F2000AB2CBB24EA18FB08FE9D9001FF9D300D01
:100F3000112463307105C9F01CEFC11613E0D1060E
:100F400050F46130710509F49ECF6230710589F06B
:100F50008E2FE32F98CF6430710571F066307105E4
:100F6000B9F3E52F9B2F8F2F8ECFEB2F852F9F2F40
:100F70008ACF852F932F87CF832FE52FF8CF8091AE
:100F80006B03823060F48170826080936B03809188
:100F90006E03873918F086E980936E0308958235D1
:100FA000B0F381708065F1CFFA01882311F00995C3
:100FB0000895FB01FCCF8091B1039091B20390930F
:100FC000200180931F010895A0E0B0E0EAEEF7E071
:100FD0000C94CA31FB018FEF9FEF4430510508F4A8
:100FE00065C04091D50341FB882780F990E0880FC8
:100FF000991F42FBAA24A0F8B12CAA0CBB1CAA0C76
:10100000BB1C8A299B2940FB882480F8912C8829C5
:10101000992943FBCC24C0F8D12C53E0CC0CDD1C27
:101020005A95E1F78C299D2944FBEE24E0F8F12C38
:1010300064E0EE0CFF1C6A95E1F78E299F2945FBC1
:10104000002700F910E075E0000F111F7A95E1F715
:10105000802B912B46FB222720F9C22F20E0D22F94
:10106000A6E0CC0FDD1FAA95E1F78C2B9D2B47FB4B
:10107000442740F920E8429FA0011124842B952B9E
:101080002091D603322F3170932B26952170B22FE9
:10109000BB0FA0E08A2B9B2B092E000CAA0BBB0BCD
:1010A00080839183A283B38380E090E0CDB7DEB7E5
:1010B000ECE00C94E631AC0123E0969587952A95F7
:1010C000E1F78E719927FC01EF52FE4F0190F081FC
:1010D000E02D4F70552721E030E002C0220F331F72
:1010E0004A95E2F7662341F0E22BF32B8F529E4F95
:1010F000DC01ED93FC93089520953095E223F323D2
:10110000F5CFE0912203F0912303309729F001906D
:10111000F081E02D0995089580E008952091CF0198
:101120003091D0012817390771F09093D001809346
:10113000CF01E0912203F0912303309721F0068044
:10114000F781E02D099508952091CD013091CE01D0
:101150002817390771F09093CE018093CD01E0916B
:101160002203F0912303309721F00084F185E02DD4
:10117000099508959C01FC0132968FEF90E0419112
:10118000461751F08F3F19F4411101C0892F9F5F1D
:101190009630A9F78F3F09F40895280F311D87FD78
:1011A0003A95F901628308952FB7F8948091C901A7
:1011B0009091CA01A091CB01B091CC012FBF0895AD
:1011C0008091B3039091B403892B91F00E94D408CD
:1011D00020912C0330912D03AC01421B530B9A013B
:1011E00081E04091B3035091B4032417350708F40C
:1011F00080E081700895CF93C82F8091D60382FF3D
:101200000CC0809170038C1741F00E94D408909319
:101210002D0380932C03C0937003CF910895A4E015
:10122000B0E0E5E1F9E00C94D4318FB7F894209167
:10123000C9013091CA014091CB015091CC01298361
:101240003A834B835C838FBF69817A818B819C81D8
:101250002496E2E00C94F0318091C801089508953D
:101260000895FC019B018091BB019091BC01861700
:10127000970740F0672B29F48091E8008E778093E0
:10128000E800C90140E0009741F4411106C0809197
:10129000E80082FF2FC080E00895209121032223DF
:1012A000A9F12530A9F12091E80023FD2DC020915E
:1012B000E80022FDECCF2091E80020FFE4CF309140
:1012C000F3002091F200009719F02830310558F012
:1012D00041E02830310509F040E02091E8002E7708
:1012E0002093E800D0CF41914093F10001972F5F08
:1012F0003F4FE9CF80912103882341F0853041F0B1
:101300008091E80083FFC3CF81E0089582E00895D3
:1013100083E008958091B50187FF13C08091E800B4
:1013200082FF06C08091E8008B778093E80004C0BC
:10133000809121038111F2CF0895809121038823A8
:10134000D9F38091E80080FFF8CF8091E8008E7794
:10135000ECCF2091E4003091E50095E6A901809161
:10136000EC008170882331F08091E80080FF06C096
:1013700080E008952091E80022FD1BC080912103A8
:10138000882391F0853091F08091EB0085FD10C0AD
:101390002091E4003091E5004217530701F391508A
:1013A0009111DCCF84E0089582E0089583E00895F0
:1013B00081E00895E8EDF0E080818E7F80831092D7
:1013C000E2001092DA001092E100A0EEB0E08C9101
:1013D00081608C9380818F77808319BCA7EDB0E00A
:1013E0008C918E7F8C9380818F7E80831092B4014C
:1013F0000895EF92FF920F931F93CF938C017B017F
:101400000E94A909C82F81110EC08091E80085FDB6
:1014100011C08091E8008E778093E8000E94A909AE
:10142000882399F3C82F8C2FCF911F910F91FF9094
:10143000EF900895F80180818093F100F1E0EF1AB8
:10144000F108E114F10479F30F5F1F4FDECF982FFD
:10145000E42FE2709093E900891308C0762F242FBF
:1014600050E0E11111C091E0980FF4CF7091EC00C1
:101470002091ED005091F00021FD06C09F5F973054
:1014800049F78093E90008953091EB003E7F309357
:10149000EB003091ED003D7F3093ED003091EB009B
:1014A00031603093EB007093EC002093ED0050938B
:1014B000F0002091EE0027FDE1CF0895A0E0B0E01C
:1014C000E4E6FAE00C94CE31C8EDD0E088818F7E5E
:1014D0008883E7EDF0E080818160808384E082BFD3
:1014E00081E08093B40188818E7F888302EE10E0D2
:1014F000F80110821092DA0081EEC82ED12CF6018C
:10150000108288818F77888388818068888388812A
:101510008F7D888319BC109221031092B301109221
:1015200008031092B20190EEE92EF12CF7018081B0
:101530008B7F808388818160888342E060E080E0E7
:101540000E94270AF60180818E7F8083F8018081C6
:1015500081608083808188608083F70180818E7FB5
:101560008083888180618883CDB7DEB7E8E00C9402
:10157000EA319C012115310509F408958FE99FE0B6
:101580000197F1F700C0000021503109F3CF81E04D
:101590008093E00080E28093D8001092C9008FE130
:1015A0009EE40197F1F700C0000087E090EBDC01BA
:1015B0008093D9039093DA03A093DB03B093DC0309
:1015C00088E19CE00FB6F894A895809360000FBE68
:1015D00090936000FFCFCF93DF93D82FC92F81E086
:1015E0008093E9008FEF9091E80095FD07C095ED9D
:1015F0009A95F1F7000081508111F5CF8091E800B4
:1016000085FD03C0DF91CF91089540E050E068E090
:1016100070E08D2F9C2F0E94F9098091E8008E7751
:101620008093E80088E0ED2FFC2FA0ECB1E0019062
:101630000D928A95E1F7E6CF8093BD017093BF01CB
:101640006093BE01809121038430F9F48093E90016
:101650008FEF9091E80095FD07C095ED9A95F1F711
:10166000000081508111F5CF8091E80085FF0DC009
:1016700040E050E063E070E08DEB91E00E94F909FA
:101680008091E8008E778093E8000895BC0183E0A4
:101690000E941C0B0895BC0184E00E941C0B08955D
:1016A000CF93682FC92F84E090E00E94C0326C2F46
:1016B00082E290E00E94C032CF910895882381F0A9
:1016C00065E283E290E00E94C03262E884E290E04A
:1016D0000E94C03262E785E290E00E94C032089525
:1016E0006FEF83E290E00E94C0326FEF84E290E0FF
:1016F0000E94C0326FEFEFCF1F93CF93DF93962FEF
:10170000122F632F8830D8F49530C8F44530B8F4E0
:10171000C42FD0E0CC0FDD1F2AE0929FC00DD11D59
:10172000112492E3899FC00DD11D1124CE0187960B
:101730000E94C032612FCE0188960E94C032DF9194
:10174000CF911F910895CF93DF93CBEDD1E060E06F
:10175000CE010E94C0322196C11584E0D807B9F7A6
:10176000DF91CF910895CF9384E090E00E94AC3256
:10177000C82F82E290E00E94AC32982F8C2FCF913C
:10178000089583E290E00E94AC32853289F484E2CD
:1017900090E00E94AC32823859F485E290E00E94D9
:1017A000AC3291E0823709F090E0892F8170089582
:1017B00080E0FCCF0F931F93CF93DF93883030F5F9
:1017C000653020F5453010F5C42FD0E0CC0FDD1F7B
:1017D0002AE0629FC00DD11D112432E3839FC00D0A
:1017E000D11D1124CE0187960E94AC32082F10E043
:1017F000102F0027CE0188960E94AC329801282B2A
:10180000C901DF91CF911F910F91089580E090E081
:10181000F8CF462F672F20911F0330912003232BF1
:1018200091F4703F39F4403F71F48091F10190914F
:10183000F2010895883038F4753028F4453018F4F2
:101840000E94DA0B089580E090E00895A0E0B0E0F7
:10185000ECE2FCE00C94CF317C01009174038091A8
:101860007303082BC7E0D0E010E0C8010C2E02C0C3
:10187000959587950A94E2F780FD09C02197A8F70E
:10188000D12C8D2DCDB7DEB7E7E00C94EB31DC2EFB
:10189000B7018C2F0E94090C0E949105019771F3EA
:1018A000F0CFCF93DF93D82FC92F0E94260C6D2F36
:1018B0007C2F0E94090C0E949105DF91CF91089521
:1018C000FC0183819481892B61F08181908189233E
:1018D0008F3F39F0808191810E94510C0E949C04BD
:1018E000089580E008951F93CF93DF93182FD92F89
:1018F000662399F0442389F00E94260CC82F682F94
:10190000812F9D2F0E94B904612F7D2F8C2F0E9463
:10191000090CDF91CF911F9108950E94F004C82F08
:10192000F3CF0F931F93CF93DF9301EB13E0C7EB3C
:10193000D1E0CE010E94AC32F80161918F0186178F
:1019400019F0CE010E94C0322196CB3DF1E0DF07B5
:1019500081F7DF91CF911F910F9108950F931F93FE
:10196000CF93DF9301EB13E0C7EBD1E0CE010E94F0
:10197000AC32F80181938F012196CB3DF1E0DF0776
:10198000A9F7C5EED6E0FE0185919491009711F07C
:10199000FC0109952C96F7E0C537DF07A1F7DF9129
:1019A000CF911F910F9108958091710390917503CC
:1019B000892B8093A40180917003882309F1809181
:1019C000B3039091B403892B29F00E94E0088111A0
:1019D0000E9443058091A40190917003892B80930C
:1019E000A40120E086EA91E0FC01308101963111EA
:1019F0002F5F31E08C3A9307B9F721110E9443051C
:101A000048E050E064E273E084EA91E00E948F32A3
:101A1000892BA9F088E0E4EAF1E0A4E2B3E00190C8
:101A20000D928A95E1F7E0912203F091230330971C
:101A300031F00280F381E02D84EA91E00995089568
:101A4000882339F090917103892B809371030E9450
:101A5000D40C0895882339F090917503892B8093D5
:101A600075030E94D40C0895882321F00E943B0541
:101A70000E94D40C0895882341F0809590917503BD
:101A80008923809375030E94D40C0895CF93C82FA7
:101A90008823A9F08CEF8C0F813A98F4E6EAF1E004
:101AA0008CEA91E02191C217B1F18E179F07D1F70F
:101AB0006C2F84EA91E00E94BA080E94D40CCF9166
:101AC000089580E28C0F883068F4C77021E030E020
:101AD00001C0220FCA95EAF780917103822B80938F
:101AE0007103EBCF8BE58C0F833038F42C2F24520D
:101AF000330BC9010E948E08E2CFC85AC731F8F6ED
:101B0000EC2FF0E0EE0FFF1FED58FE4F808191812A
:101B10000E94A408D4CF8C2F0E942E050E94D40CC2
:101B2000C7CFCF93DF93EC01805E9109089720F037
:101B30006AE27DE0209711F460E27DE0CE010E9430
:101B400070048C2F0E94460DDF91CF91089566237B
:101B500029F0209175032260209375039C01305673
:101B6000211540E2340720F0305E2115304108F4A1
:101B700099270E94910D0895882339F19CEF980FC1
:101B8000913A28F40E942E050E94D40C089590E208
:101B9000980F983050F4877091E001C0990F8A95A2
:101BA000EAF7892F0E943B05EFCF9BE5980F933012
:101BB00028F480E090E00E948E080895885A8731CA
:101BC00020F480E090E00E94A4080895CF93DF9372
:101BD000EC010E94BC0DCE01805E9109089720F0B7
:101BE0006BE37DE0209711F464E37DE0CE010E9479
:101BF0007004DF91CF9108950F931F93CF93C82F57
:101C00000091D1031091D203893321F00091CF03C9
:101C10001091D0038C2F0E94460D0115110539F447
:101C20008C2F0E94BC0DCF911F910F9108958FE9C9
:101C30009FE00197F1F700C0000001501109EDCFBE
:101C40000F931F93CF93DF93C62FD42F122F882388
:101C5000A9F0609365030E94D4089093B00180932B
:101C6000AF01C77081E001C0880FCA95EAF70E94F2
:101C7000200DDF91CF911F910F9108958091650301
:101C800068133DC02091AF013091B0014FB7F89477
:101C90008091C9019091CA01A091CB01B091CC0172
:101CA0004FBF821B930B883C910548F56D130CC008
:101CB000812F0E94FC0DD77081E001C0880FDA955A
:101CC000EAF70E94340DD5CFC77001E0802F01C024
:101CD000880FCA95EAF70E94340D80E28D0F883094
:101CE00050F48D2F877001C0000F8A95EAF7802F7E
:101CF0000E94200DDDCF812F0E94FC0DBACFC7704E
:101D000081E001C0880FCA95EAF7DBCFA0E0B0E020
:101D1000ECE8FEE00C94CF31EC019881992309F4B2
:101D20009CC09130E1F599818A81913021F422960D
:101D30000E94FC0D05C0923029F422960E94460DA7
:101D40002196EBCF933021F422960E94BC0DF8CF60
:101D5000943011F02196F4CF229620E030E06AE032
:101D6000AE014F5F5F4F8053990B8A30910560F051
:101D70002115310529F38FE99FE00197F1F700C0A4
:101D8000000021503109F4CF629FF001639FF00DF4
:101D900011249C012E0F3F1F8981EA01E1CFE92F19
:101DA000F0E0E252FE4FD490292F269526952695F5
:101DB00030E0F901E253FE4F84919770F901E2544B
:101DC000FE4FE490F12C092E02C0F594E7940A949A
:101DD000E2F741E0E422FF24F901E255FE4F0491CD
:101DE00010E0092E02C0159507950A94E2F70170DC
:101DF0001127E82FF0E002C0F595E7959A95E2F7F4
:101E0000E0FD0CC0E114F104A1F48D2D0E94FC0D45
:101E10000115110509F494CF8CE28ACF81EE0E945E
:101E2000460DE114F10479F48D2D0E94FC0D81EE34
:101E300007C086EE0E94460D8D2D0E94FC0D86EE99
:101E40000E94BC0DE5CF86EE0E94460D8D2D0E94AE
:101E5000FC0D86EE0E94BC0DEACFCDB7DEB7E7E001
:101E60000C94EB3180E090E00E948E0880E090E0DE
:101E70000E94A408109275030E94D40C0895109239
:101E80007103E6EAF1E086E0DF011D928A95E9F749
:101E90000E94320F08950E943F0F2FEF84E39CE0D1
:101EA000215080409040E1F700C0000088E19CE0B4
:101EB0000FB6F894A895809360000FBE90936000D1
:101EC000FFCFCF92DF92EF92FF92FB018FEF9FEF58
:101ED0004430510508F47FC0C080D180E280F38097
:101EE0000E943F0FD701C601B695A7959795879594
:101EF0008170282F220FD701C60181709927AA2748
:101F0000BB27822BB701A60132E0769567955795DE
:101F100047953A95D1F74170440F440F842BB70190
:101F2000A601E3E07695679557954795EA95D1F731
:101F30004170440F440F440F842BB701A601F4E015
:101F40007695679557954795FA95D1F741704295E3
:101F5000407F842BB701A601A5E07695679557953C
:101F60004795AA95D1F741704295440F407E842B46
:101F7000B701A601B6E07695679557954795BA954E
:101F8000D1F741704295440F440F407C842BB70138
:101F9000A60197E076956795579547959A95D1F75D
:101FA000479544274795842B8093D503D1FA8827FA
:101FB00080F9880F9D2D9170892B9091D6039C7F7D
:101FC000892B8093D6038091D5039091D6030E94EC
:101FD000500B80E090E0FF90EF90DF90CF9008955D
:101FE000E1EBF3E0128E138E8FEA90E09183808311
:101FF00085E0848F28E833E13383228322E330E0D5
:10200000378B268B28EC30E0318F208F158E178E82
:10201000168E20E530E031A320A382A30E94910C0C
:102020000E943F0F1092D6031092D50380E0846087
:102030008093D60380E094E00E94500B0E94AE0C87
:1020400008958F929F92AF92BF92CF92DF92FF92AC
:102050000F931F93CF93DF938090210190902201E3
:1020600081E090E09093220180932101A12CB12C7A
:1020700000E0650110E013C0FE01259134914F2D61
:10208000612F802F0E947C0B2296F39485E0F8123A
:10209000F3CF85E0C80ED11C1F5F153039F0E60183
:1020A000CC0FDD1FCF5DDC4FF12CE6CF0F5F89E158
:1020B000A80EB11C0830E9F60E94F00F90922201A0
:1020C00080922101DF91CF911F910F91FF90DF90BE
:1020D000CF90BF90AF909F908F90089580E00E9426
:1020E0005E0B60E086E290E00E94C0320E94211008
:1020F0000E94A30B81E00E945E0B0895AAE2B0E06B
:10210000E4E8F0E10C94D33185EB91E0FC01019619
:102110002091F100208321E08D3B9207B9F7809157
:10212000B601893009F456C0C8F4823009F4B3C04E
:10213000833009F482C0813071F18091E80083FF1F
:10214000E7C08091B5019091B6019A3008F0E0C0E7
:10215000E92FF0E0E75AFC4C0C94A8318A3009F4DE
:1021600089C08B3051F78091B501813231F7809170
:10217000B9019091BA01892B01F78091E800877F1E
:102180008093E8000E948A098091B701809304013E
:102190000E943F0FD2CF8091B501813A71F68091B4
:1021A000E800877F8093E8008091B9019091BA019F
:1021B000892B61F060E080E090E070E00E943109DE
:1021C0008091E8008B778093E800B7CF68E080ECDF
:1021D00091E0F3CF8091B501813209F0AECF8091CB
:1021E000B9019091BA018D7F892B09F0A6CF80911A
:1021F000E800877F8093E8008091E80082FF18C0A4
:102200009091F3008091F200029731F48091F100F7
:10221000813011F0863021F48091F1008093C80163
:102220008091E8008B778093E8000E948A0985CF2F
:10223000809121038111E0CF80CF8091B501813A57
:1022400009F07BCF8091B9019091BA01892B09F0F7
:1022500074CF8091E800877F8093E8008091E80048
:1022600080FFFCCF809104018093F1008091E80011
:102270008E77D9CF8091B501813209F05ECF809100
:10228000E800877F8093E8000E948A098091B80166
:102290008093B10152CF8091B501813A09F04DCFC1
:1022A0008091E800877F8093E8008091E80080FFBC
:1022B000FCCF8091B101D8CF803889F0823841F5C8
:1022C0008091B9018F70873018F58093E900809173
:1022D000EB0085FB882780F91092E90006C0809109
:1022E000B20190910803911182609091E800977F6C
:1022F0009093E8008093F1001092F1008091E80043
:102300008E7723C0811116C08091B701813011F101
:102310008091E80083FF0AC08091E800877F809366
:10232000E8008091EB0080628093EB00AA96E3E0E6
:102330000C94EF31823061F78091B701882389F0E6
:102340001092E9008091E800877F8093E8000E9466
:102350008A09DECF81E0933009F080E080930803A2
:10236000EFCF8091B9018F702FEF280F263080F6C4
:102370008093E9002091EB0020FFE2CF933031F40D
:102380008091EB0080628093EB00DACF9091EB00BC
:1023900090619093EB0021E030E0A90102C0440F6E
:1023A000551F8A95E2F74093EA001092EA00809167
:1023B000EB008860E8CF8111ABCF1091B7011F7798
:1023C0008091E3008078812B8093E3008091E80086
:1023D000877F8093E8000E948A098091E80080FF4F
:1023E000FCCF8091E30080688093E30083E01111CB
:1023F00001C082E0809321038BCF8058823008F0A7
:1024000087CF4091B7015091B8014C3D83E0580708
:1024100099F583E08A838AE289834FB7F894DE01D5
:10242000139620E03EE051E2E32FF0E05093570096
:10243000849120FF03C082958F703F5F8F708A3038
:10244000C8F0895C90E08D939D932F5F243161F7F4
:102450004FBF8091E800877F8093E8006AE270E0D8
:10246000CE0101960E9431098091E8008B7780931C
:10247000E8004ECF805DE6CF8091B9019091BA011E
:10248000252F33272330310509F44AC078F5213050
:10249000310509F483C08BE590E0EEE5F2E02230EF
:1024A000310509F035CF2091E800277F2093E8001F
:1024B0002091BB013091BC018217930708F49C0165
:1024C00040E02115310509F06EC041116CC08091CA
:1024D000E80082FDC9CF80912103882329F285304D
:1024E00019F28091E80083FFF2CFBECF213231058F
:1024F00009F445C02232310509F00ACF8330910535
:1025000008F006CFFC01EE0FFF1FEC5CFE4F0190C0
:10251000F081E02D8F5C9E4FDC018C9190E010C02B
:10252000CA019927423019F18330910568F4892B4B
:10253000B1F4EDE1F3E0E4918E2F90E0EDE1F3E012
:10254000009709F4E5CEAFCF039709F0E1CEEBECAD
:10255000F2E0E4918E2F90E0EBECF2E0F1CFE1E0DD
:10256000F3E0E4918E2F90E0E1E0F3E0E9CFE9EED3
:10257000F2E0E4918E2F90E0E9EEF2E0E1CF8330DB
:10258000910508F0C5CEFC01EE0FFF1FE65CFE4F83
:102590000190F081E02D89E090E085CF82E190E02C
:1025A000E9EBF2E080CF80912103882309F45CCF2E
:1025B000853009F459CF8091E80083FD55CF809193
:1025C000E80082FD84CF8091E80080FF7ACF90916F
:1025D000F3008091F2002115310519F08830910542
:1025E00050F041E0089709F040E08091E8008E77D4
:1025F0008093E80066CF44914093F10031962150DA
:1026000031090196E8CF803809F082CE8091E80048
:10261000877F8093E8008091B3018093F1006ECEB4
:10262000811176CE1091B701123008F071CE8091F1
:10263000E800877F8093E8001093B3010E948A0925
:102640001123D1F084E08093210342E061EC81E02A
:102650000E94270A42E261EC84E00E94270A42E2DB
:1026600061EC82E00E94270A42E260EC83E00E9473
:10267000270A809121034CCE8091E30087FDE2CFB1
:1026800081E0E1CF809373030E94320F089580911F
:102690002301877F80932301909175039D7F909301
:1026A000750384FF08C08F7E80932301809171039E
:1026B0008260809371038091230185FF08C08F7D24
:1026C00080932301809171038062809371030E9443
:1026D000D40C0895CF92DF92FF920F931F93CF9364
:1026E000DF93EC018B01F42E8091230182FF6BC0FC
:1026F000C0905D03D0905E03CC16DD0619F02097E4
:1027000009F061C0809123018B7F80932301C1E098
:1027100081FD10C080915B0390915C039801281BA0
:10272000390BC1E080911F019091200128173907D2
:1027300008F4C0E0C17080912301C0FB81F980934F
:1027400023016C2FC6010E945B088091710381FFF9
:1027500008C08091230180618093230182E00E9460
:102760003B058091710385FF08C080912301806241
:102770008093230180E20E943B056C2FC6010E94DA
:10278000A70DFF2031F08091CC0385FF02C086FFAA
:1027900033C08091CF039091D0030E94B90A8091F9
:1027A0005D0390915E039C013056211540E2340791
:1027B00020F0305E2115304108F499270E94E60D83
:1027C0000E94471315C0CE019056811520E2920752
:1027D00020F0905E81159041B8F4CE0199270E94B7
:1027E000E60D80915D0390915E03C817D90741F310
:1027F00010935C0300935B03DF91CF911F910F91C6
:10280000FF90DF90CF900895CE01E9CF0F931F93F3
:10281000CF93DF938B01D82FC92F0E94BF07A80148
:102820006D2F7C2F88E090E00E94D232DF91CF9113
:102830001F910F910895EBE6F3E083E0808311820E
:102840008FEF828386E98383148263E070E08FEFE9
:1028500096E90E9406140895A4E0B0E0E2E3F4E1F2
:102860000C94D43180916F03833018F48F5F809380
:102870006F0380916B0390916C03A0916D03B091F5
:102880006E03BC01CD010E9406142496E2E00C9474
:10289000F031A4E0B0E0EFE4F4E10C94D4318091A5
:1028A0006F03882319F0815080936F0380916B032D
:1028B00090916C03A0916D03B0916E03BC01CD01AA
:1028C0000E9406142496E2E00C94F03168EE7EEF4C
:1028D00080E090E00E94DE3260E082E090E00E94C2
:1028E000C03260E083E090E00E94C0321092730337
:1028F00060E084E090E00E94C03264E082E290E018
:102900000E94C03260E085E090E00E94C03260E04A
:1029100086E090E00E94C0326FEF87E090E00E9476
:10292000C03240E050E0BA0188E090E00E94D2322C
:1029300060E08DE090E00E94C03240E050E0BA01DB
:1029400088E190E00E94D23260E087E190E00E944E
:10295000C03240E050E0BA018CE190E00E94D232F7
:1029600060E070E080E290E00E94DE3240E050E003
:10297000BA0188E190E00E94D23280E00E945E0BB2
:102980000E946E1040E050E0BA018FE090E00E949B
:10299000D23240E050E0BA0183E190E00E94D232AE
:1029A0000895A5E0B0E0E7EDF4E10C94C731809123
:1029B0006B0380FD0AC0EAE9F2E011821082128204
:1029C000339622E0ED3FF207C1F780900303909029
:1029D00004038114910409F465C0809107038111F7
:1029E00061C050906E03A12CB12C66246394712CAD
:1029F0002091690330916A03C3010A2C02C0880F39
:102A0000991F0A94E2F782239323892B09F43FC08C
:102A1000F401E590F490E114F10409F443C045E0B9
:102A200050E0B701CE0101960E94793289818F3F33
:102A300071F12A8190E0280F392F311D22323105A2
:102A400014F021E230E06901CC0CDD1CC20ED31E73
:102A5000960126563D4F69018C01000F111F080F8A
:102A6000191F06561D4F0C151D0520F055E0E50EEB
:102A7000F11CD5CF452D36E9351508F446E9980106
:102A80006C818B810E9433070D5F1F4FECCF82E07A
:102A9000880E911C9FEFA91AB90A29E0A216B10469
:102AA00009F0A6CF559A3BB13F7D2BB120624FB7BD
:102AB000F8948AE992E0FC010196508168E02BB914
:102AC000000000C057FF3BB9550F000000C000C018
:102AD00000C03BB900C06A9591F752E08D3F950761
:102AE00051F74FBF8FE594E00197F1F700C0000068
:102AF0002596EFE00C94E331EF92FF921F93CF9372
:102B0000DF93EC018AE9E82E82E0F82E10E0409194
:102B10006E03473908F046E98C81970160916D0397
:102B2000810F0E943307195F83E0E80EF11C173E06
:102B300071F70E94D1149A818C8190FF08C08F5F39
:102B40008C83DF91CF911F91FF90EF90089581507A
:102B5000F7CFA0E0B0E0EFEAF5E10C94CE31FC0154
:102B60008281DD24D39480FF02C0DD24DA940AE957
:102B700012E0C0E0D0E0F80111821082128294E0ED
:102B8000E92EF12CC12C809199028C0D8232ECF14E
:102B900061E20E947231892F082E000C990B8C176C
:102BA0009D07A9F480916E038E9DA0018F9D500D0D
:102BB00011245595479555954795473908F046E9AD
:102BC000980160916D0380916C030E943307CD0CD6
:102BD000F1E0EF1AF108E114F104A9F621960D5F76
:102BE0001F4FC132D10539F60E94D114809199024C
:102BF00091E0D9120EC0882391F081508093990200
:102C0000CDB7DEB7E8E00C94EA3187FFC5CF8F5D22
:102C1000C3CF90E00196BE010E949431EFCF80E2D5
:102C2000EDCF0F931F93CF93DF93CAE9D2E0FE015C
:102C3000118210821282339682E0ED3FF807C1F7CD
:102C400000E010E080919802082E000C990B081704
:102C50001907A4F180910701082E000C990B801729
:102C6000910764F140916E03473908F046E99E01EF
:102C700060916D0380916C030E9433070F5F1F4FBB
:102C8000239601321105F1F60E94D11480910601BC
:102C900090919802980F9093980220910701280F25
:102CA00020930701121614F490321CF08195809342
:102CB0000601DF91CF911F910F910895198218821B
:102CC0001A82DCCFAEE0B0E0E8E6F6E10C94CE315B
:102CD0008D879E87AD85BE8514961C91212F30E08F
:102CE000D9010E9448339B01AC010E9413336983D0
:102CF0007A838B839C83E0E2F0E0E11BF109A5E598
:102D0000B0E09B01AC010E94133369877A878B87FF
:102D10009C879F01DF010E94B5319B01AC010E949D
:102D20001E336D837E838F8398879B01AC018981DD
:102D30009A81AB81BC81280F391F4A1F5B1F6985AF
:102D40007A858B859C850E942633022F30E00A32DB
:102D5000E0F5C901880F991F820F931F95958795FC
:102D6000182F10953AE9C32E32E0D32EF12C85E5C9
:102D7000E82EE01A8E2DF1FC802F412F173908F034
:102D800046E9960160916D030E943307F394B3E026
:102D9000CB0ED11CE1E2FE12EDCF0E94D114AD8525
:102DA000BE8514969C9181E0992319F0903219F414
:102DB0008FEF8093050180910501890FED85FE85D8
:102DC00084832E96E8E00C94EA3185E590E0DC01FE
:102DD000A21BB30BCD01880F991F8A0F9B1F97FF72
:102DE000BDCF0196BBCF90916B0390FF0CC0EAE979
:102DF000F2E0818360834283339692E0ED3FF907EE
:102E0000C1F70E94D1140895A3E0B0E0EAE0F7E131
:102E10000C94D43190916B0390FF0DC0473908F0AA
:102E200046E99E012F5F3F4F0E9433074B81698126
:102E30008A810E94F3162396E2E00C94F031CF933E
:102E4000DF93EC01EC81F0E0EF54FB4F4491EBE6B3
:102E5000F3E0628181810E9404178C818F5F8C83F3
:102E6000DF91CF910895CF93DF93EC01EBE6F3E090
:102E7000438162818C810E9404178C818F5F8C83D7
:102E8000DF91CF910895A7E0B0E0E9E4F7E10C9479
:102E9000C731E82E762EF42E622E90916B0390FFB0
:102EA00030C0E92FE695AE2FB0E0A05CBE4F8C910C
:102EB000809367039E7F923041F586E9841708F47A
:102EC00046E99E012F5F3F4F672D8E2D0E943307ED
:102ED0004B8169818A810E94F316E0926C037092A3
:102EE0006D03F0926E03662061F080916B03909108
:102EF0006C03A0916D03B0916E03BC01CD010E94E3
:102F000006142796EFE00C94E331823019F4F09028
:102F10006E03E3CF863019F4E0906C03DECF893086
:102F2000D9F38931D1F6E9519E2F9170592EE6954A
:102F3000F0E0EF54FA4FE4910E2F10E08AE9C82E2A
:102F400082E0D82EA12CB12C91E2892E912CC501C2
:102F5000B4010E9480318E2D511017C0860F4F2D65
:102F6000A6E9AF1508F446E99601672D0E943307DC
:102F7000A00EB11EB3E0CB0ED11C8DEFC81682E0BF
:102F8000D80629F70E94D114A8CF861BE8CFEBE61C
:102F9000F3E0818121E043816281885F0E944317D1
:102FA0000895EBE6F3E0818121E04381628188505E
:102FB0000E9443170895EBE6F3E0628128E0620F78
:102FC00008F46FEF21E0438181810E944317089547
:102FD000EBE6F3E0628128E0621B08F460E021E0A8
:102FE000438181810E9443170895EBE6F3E043811A
:102FF00028E0420F08F44FEF21E0628181810E94B6
:1030000043170895EBE6F3E0438128E0421B08F400
:1030100040E021E0628181810E9443170895A0E091
:10302000B0E0E5E1F8E10C94C831FC0182806480F5
:1030300081E08483E1EBF4E09490E0E3F5E0E49157
:10304000C3EFD1E09AE9E92E92E0F92E28E9C22EE9
:1030500022E0D22E32E0A32EBB24B39477247A94BC
:10306000E9190E2F10E082E0881530F080916C0392
:10307000888380916D038983611019C01B821A8235
:103080004A81473908F046E99701698188810E94A1
:103090003307259683E0E80EF11CCC16DD0619F700
:1030A0000E94D114CDB7DEB7EEE00C94E4318B81F1
:1030B0008823E9F081508B83789EC00111246C81B4
:1030C00070E00E948031FB01FF27EF54FB4F849199
:1030D000E82FE9197E9EC0011124B8010E948031B9
:1030E00080916E03689FB00111247A83C9CF0E943A
:1030F0006932AC0190916E03969591589A9D90011A
:103100009B9D300D1124232F3327421753070CF0BA
:10311000B7CF82E0881590F40E9469326FEF70E0BB
:103120000E94943188830E94693220916D03269514
:10313000622F70E00E949431280F29831A828091B7
:103140006E03893C20F088EC8C838B8399CF84318B
:10315000D8F784E1F9CF60916B03669570E04BE09E
:1031600050E088E091E00E948232892B19F481E0DE
:10317000809368030E94D4089093120380931103F4
:103180000895A4E0B0E0E7ECF8E10C94D43190911C
:103190006B0390FF34C08823B1F18932B0F58F778B
:1031A000880F90916B039170892B80936B0366233A
:1031B00061F080916B0390916C03A0916D03B091CD
:1031C0006E03BC01CD010E94061460916B036695ED
:1031D00070E04BE050E088E091E00E948232892B61
:1031E000B1F01092680381E08093140320E04091D5
:1031F0006E0360916D0380916C030E9443172496C7
:10320000E2E00C94F03181E0CBCF88E2C9CF0E949C
:10321000AB18E9CF80916B0386958F5F893208F0F8
:1032200081E061E00E94C118089590916B0396952A
:103230008FEF890F913009F488E261E00E94C11894
:10324000089521E030E0A90102C0440F551F8A957E
:10325000E2F7CA012091690330916A036623B1F055
:10326000242B352B30936A032093690380916803E4
:10327000811106C080916B0360E086950E94C118A1
:1032800080916B0380FF0E94D114089580959095E2
:1032900028233923E7CF1F93CF93DF93182F0E9462
:1032A0008108682F617080E00E942119111121C0EE
:1032B00060E081E00E94211960E082E00E94211913
:1032C00060E083E00E94211960E084E00E942119FF
:1032D00060E085E00E94211960E086E00E942119EB
:1032E00060E087E00E942119812FDF91CF911F912B
:1032F0000895C12FD0E0BE0175956795617081E09A
:103300000E942119BE017595679575956795617045
:1033100082E00E942119BE0123E0759567952A95E8
:10332000E1F7617083E00E942119BE0134E07595D8
:1033300067953A95E1F7617084E00E942119BE011A
:1033400045E0759567954A95E1F7617085E00E94C3
:103350002119BE0156E0759567955A95E1F76170A0
:1033600086E00E942119CC0FCD2FCC1FDD0B6C2FD6
:103370006170B7CF0E944B19809374030E94320F83
:10338000089521E030E001C0220F8A95EAF780918C
:103390007403822B0E94BA1908959091D60392FF6C
:1033A00010C098E0899F90011124622B60937603EE
:1033B0000E94C1190E94D4089093780380937703E8
:1033C00008950E94C119089521E030E0A90102C0CA
:1033D000440F551F8A95E2F7CA01809590917403B6
:1033E00089230E94BA19089520917603809582233B
:1033F00080937603982F9770911117C030E0482F73
:10340000082E000C550B2417350779F09091D60340
:1034100092FF0BC08595859585950E94E4191092C1
:103420007603109278031092770308959091D60353
:1034300092FB222720F9281769F080FB92F99093DC
:10344000D6038091D5039091D6030E94500B82E061
:103450000E94F419089580917403982F9670963005
:1034600021F488600E94BA190895877FFBCF682FE6
:10347000617080E00E942119089590916B0390FF84
:1034800008C09695981728F0961718F40E940A1904
:10349000089561E00E94C1180895A0E1B0E0E3E55D
:1034A000FAE10C94C4312C01DC019C9111968C91B1
:1034B000119713962D913C911497232B09F4CFC0AB
:1034C00089238F3F09F4CBC041E012966C9112978B
:1034D0008D919C910E94730C1C01F201F281FD8779
:1034E000815095458F3F910508F043C0410125E586
:1034F0009226F111B9C0A0E48A16910408F0C4C361
:10350000A0903A03B0903B03C0903C03D0903D03A1
:10351000E0903E03F0903F03E0914003109141039F
:1035200021E030E040E050E060E070E080E090E0DA
:10353000082D0E94FB31A222B322C422D522E6220A
:10354000F722082F0E2319230E94143209F476C0A3
:10355000A0E12A16AFE53A0609F462C4B1E12B16E0
:10356000BFE53B0609F038C3FD85F111DDC382E0FC
:1035700061C4AD85AA2309F41DC3BFEF2B16310426
:1035800009F008F470C0EAE22E16EDE53E0609F4F3
:103590004FC010925A03C10182519F45409708F0D5
:1035A000B7C38FEF93E00E94AC32811147C0AEEEFB
:1035B0002A0E0BED11E02110C0C3809124019091DF
:1035C0002501A0912601B091270189839A83AB83BD
:1035D000BC837801EFEFEE1AFE0AC8010E94AC32FC
:1035E00089831A82882351F1813009F013C468015C
:1035F000F2E0CF0ED11CC7010E94AC32F82E8A83B4
:103600008823E1F0C6010E94AC32E82E8FEF8F0DC7
:10361000833008F0A0C3EB82EE2021F0CE010196AA
:103620000E94860E680123E0C20ED11C8601D1CF14
:1036300080915A0391E0892780935A038091760301
:103640008770882361F0D20112968C91882339F01B
:103650008091D60382FF03C082E00E94F419609635
:10366000E2E10C94E031410180915A03882309F48E
:10367000F4C010925A03F0EC8F16910408F040C089
:1036800020E88216910408F0B2C0840100541109A8
:103690000034110508F478C021E030E040E050E04B
:1036A00060E070E080E090E0082D0E94FB31E09146
:1036B0003A032E2BE0913B033E2BE0913C034E2B33
:1036C000E0913D035E2BE0913E036E2BE0913F03C2
:1036D0007E2BE09140038E2BE0914103E92B209358
:1036E0003A0330933B0340933C0350933D03609374
:1036F0003E0370933F0380934003E093410335C042
:1037000021E030E040E050E060E070E080E090E0F8
:103710008401005C11090E94FB31E09152032E2BC1
:10372000E09153033E2BE09154034E2BE09155035F
:103730005E2BE09156036E2BE09157037E2BE091B8
:1037400058038E2BE0915903E92B209352033093B9
:10375000530340935403509355036093560370935F
:10376000570380935803E09359038091CC0380FD65
:1037700064C38D85F8ED8F16FCE59F0609F0DBC468
:1037800027E245EE65EEE5C421E030E040E050E0A0
:1037900060E070E080E090E00E94FB31E091420345
:1037A0002E2BE09143033E2BE09144034E2BE091FE
:1037B00045035E2BE09146036E2BE09147037E2B81
:1037C000E09148038E2BE0914903E92B20934203BB
:1037D000309343034093440350934503609346035F
:1037E0007093470380934803E0934903BECF21E0E1
:1037F00030E040E050E060E070E080E090E0840184
:10380000005811090E94FB31E0914A032E2BE091F0
:103810004B033E2BE0914C034E2BE0914D035E2B6E
:10382000E0914E036E2BE0914F037E2BE09150030D
:103830008E2BE0915103E92B20934A0330934B03E5
:1038400040934C0350934D0360934E0370934F038A
:1038500080935003E093510388CF40E48416910491
:1038600008F066C0A0913A03AD83B0913B03BE83DC
:10387000E0913C03EF83F0913D03F887A0913E0374
:10388000A987B0913F03BA87E0914003EB87F0919D
:103890004103FC8721E030E040E050E060E070E070
:1038A00080E090E0082D0E94FB3139014A01B62FDB
:1038B000A72FF82FE92FAD80A222BE80B720CF809E
:1038C000C422D884D920E984E622FA84F7220B8521
:1038D00008231C8519230E94143209F027C2609422
:1038E000709480949094B095A095F095E0952D817A
:1038F00062224E8174225F81852288859822998573
:10390000B9232A85A2234B85F4235C85E5236092A5
:103910003A0370923B0380923C0390923D03B09334
:103920003E03A0933F03F0934003E093410386CE10
:1039300020E88216910408F068C0A0914203AD838C
:10394000B0914303BE83E0914403EF83F0914503BC
:10395000F887A0914603A987B0914703BA87E09101
:103960004803EB87F0914903FC8784010054110957
:1039700021E030E040E050E060E070E080E090E086
:103980000E94FB3139014A01B62FA72FF82FE92FEA
:10399000AD80A222BE80B720CF80C422D884D92097
:1039A000E984E622FA84F7220B8508231C85192373
:1039B0000E94143209F0BAC160947094809490947B
:1039C000B095A095F095E0958D8168229E81792231
:1039D0002F818222488594225985B5238A85A82380
:1039E0009B85F9232C85E223609242037092430366
:1039F0008092440390924503B0934603A0934703FB
:103A0000F0934803E093490319CE20EC8216910409
:103A100008F068C0A0914A03AD83B0914B03BE8308
:103A2000E0914C03EF83F0914D03F887A0914E0392
:103A3000A987B0914F03BA87E0915003EB87F091CB
:103A40005103FC8784010058110921E030E040E077
:103A500050E060E070E080E090E00E94FB313901CE
:103A60004A01B62FA72FF82FE92FAD80A222BE80E2
:103A7000B720CF80C422D884D920E984E622FA84F2
:103A8000F7220B8508231C8519230E94143209F0A4
:103A90004DC16094709480949094B095A095F095E9
:103AA000E0954D8164225E8175228F818822988500
:103AB00099222985B2234A85A4235B85F5238C8529
:103AC000E82360924A0370924B0380924C039092D9
:103AD0004D03B0934E03A0934F03F0935003E09334
:103AE0005103ACCDA0915203AD83B0915303BE837B
:103AF000E0915403EF83F0915503F887A0915603AA
:103B0000A987B0915703BA87E0915803EB87F091EA
:103B10005903FC878401005C110921E030E040E09A
:103B200050E060E070E080E090E00E94FB313901FD
:103B30004A01B62FA72FF82FE92FAD80A222BE8011
:103B4000B720CF80C422D884D920E984E622FA8421
:103B5000F7220B8508231C8519230E94143209F0D3
:103B6000E5C06094709480949094B095A095F09581
:103B7000E0959D8169222E8172224F818422588591
:103B800095228985B8239A85A9232B85F2234C8514
:103B9000E4236092520370925303809254039092F4
:103BA0005503B0935603A0935703F0935803E09343
:103BB000590344CD5FEF2516310409F008F462C0C3
:103BC00080E128168FE5380609F433C191E1291602
:103BD0009FE5390609F4CBCC8091CC03410180FDEF
:103BE0002CC14101D20112968C91B3EF8B16BCE52A
:103BF0009B0609F409C308F4BDCD55EF85165CE5B5
:103C0000950609F4A3C327E245EE66EE96EF891602
:103C10009CE5990609F49DC227E245EE64EEA4EF07
:103C20008A16ACE59A0609F494C2882309F4C8C23E
:103C300010926503B1E68B16BDE59B0609F4B9C386
:103C400008F08CC3F6E18F16FCE59F0608F062C110
:103C500022E082162CE5920608F489C10E94B30B7B
:103C60009093D6038093D503F401E350FC458091F3
:103C7000D5038160E331F10508F0A3C3ED59FC4C95
:103C80000C94A831410137CCB0E88B169104A0F414
:103C9000A0904203B0904303C0904403D0904503EA
:103CA000E0904603F0904703E091480310914903E8
:103CB000F0E48F1A910834CC20EC82169104A0F421
:103CC000A0904A03B0904B03C0904C03D0904D039A
:103CD000E0904E03F0904F03E09150031091510398
:103CE00040E8841A91081CCCA0905203B090530372
:103CF000C0905403D0905503E0905603F0905703C2
:103D0000E09158031091590350EC851A910808CCA2
:103D100080E128168FE5380609F485C091E129165F
:103D20009FE5390609F058CF82E07EC0C10182517B
:103D30009F45409708F00CCC34CC0115B4E01B072C
:103D400009F47CCCC8010E94AC320F5F1F4F811177
:103D5000F4CF2A9430CC8BEF8F0D833090F568012F
:103D600043E0C40ED11CEB82EE2009F45FCCC60107
:103D70000E94AC328C838823D9F0CB80DC8051E068
:103D8000C5165FEFD50610F0DC2CCC2486E0F816C3
:103D9000A1F097E0F91649F0C6010E94AC28809185
:103DA000CF039091D0030E94B90AC6010E94D02887
:103DB0006801A4E0CA0ED11C39CCC6010E94AC280F
:103DC000F7CFB4E0FB1232CC6801E4E0CE0ED11C98
:103DD000C80103960E94AC32EE2009F42FCC882350
:103DE00009F42CCC8150990B4FEF489F9001499FCB
:103DF000300D11244E2D4150550B240F351F2150ED
:103E0000310908F413CC8FE99FE00197F1F700C066
:103E10000000F5CFCE0101960E94860E670106CC08
:103E2000ED85EE2331F081E00E94C1190E942B1A2A
:103E300005CC81E00E94E419F9CF0E94D4087C01EE
:103E4000D20112968C911297882309F422C1809195
:103E5000230182FF06C040E0B70180E090E00E94AD
:103E60006A13BBE18B16BCE59B0619F1ECE18E16DB
:103E7000ECE59E0609F43CC0FAE18F16FCE59F06CE
